:10000000830100308A0004282030840021300F2032
:1000100083010A128A117B2904068001840A0406DE
:10002000031900340C2883120313C600C71B2128B0
:10003000471B292847088A004608C60A0319C70A29
:1000400082008313471883174608C60A84000008F5
:10005000080067346F346F34643420346D346F3487
:1000600072346E3469346E346734203476346934D3
:10007000653474346E3461346D34003474346534F2
:100080006D3470343D3425346434203443340034CA
:040090003F340034C5
:10009C008316031386118312861183168715071690
:1000AC00803094002830831294000930831693001A
:1000BC0083121308A500031383120800831603137D
:1000CC00111468288316031311186D286E286828DC
:1000DC00831203138C119A30930074288312031328
:1000EC008C1D79287A287428831203138C119301A0
:1000FC007F28831203138C1D842885287F28831660
:10010C000313911489288316031391188E288F28B2
:10011C008928831203138C119B309300952883122A
:10012C0003138C1D9A289B289528831203138C117A
:10013C0083169115A12883160313141CA628A7282F
:10014C00A128831203131308A50083161116AE28D9
:10015C0083160313111AB328B428AE288312031381
:10016C002508B828031383120800F03083160313F4
:10017C0088050E309F00F13085058312051185111D
:10018C000F300A128A1599270A128A110330880037
:10019C008514851005300A128A1599270A128A11BE
:1001AC00851485102130A500DC28DC28831203136C
:1001BC00A50BE128E228DB28831203138514851094
:1001CC0005300A128A1599270A128A110230880002
:1001DC00851485100D30A500F428F4288312031320
:1001EC00A50BF928FA28F32828300A128A15BB2700
:1001FC000A128A1108300A128A15BB270A128A11B0
:10020C000F300A128A15BB270A128A1106300A12FD
:10021C008A15BB270A128A1103138312080083164E
:10022C000313111419298316031311181E291F29DE
:10023C001929831603139112111783128C11C430D0
:10024C0093002829831203138C1D2D292E2928296C
:10025C00831203138C118316111B35293829831231
:10026C0086153A29831286118316031311178312EC
:10027C008C1193014129831203138C1D46294729A4
:10028C004129831203138C118316111B4E295129FA
:10029C0083128615532983128611831603131117A3
:1002AC0083128C11153093005B29831203138C1D60
:1002BC00602961295B29831203138C118316111B8E
:1002CC0068296B29831286156D2983128611831672
:1002DC00031311171115722983160313111977299A
:1002EC00782972290313831208000A128A114E20EE
:1002FC000A128A110A128A11BB200A128A110A12D6
:10030C008A1572270A128A110A128A1164200A129B
:10031C008A11A20040300A128A1564270A128A1127
:10032C003E30A6000030A7002208F000F101F01BBF
:10033C00F1037008A3007108A4002330A5000A1271
:10034C008A114C250A128A110618AD29AE29C22928
:10035C002018B129B229C1290530A5000330A60007
:10036C002930A7000030A80000300A128A11DB23C4
:10037C000A128A112014C529831203132010831228
:10038C000313051ACA29CB29E529A018CE29CF2990
:10039C00E4290A128A1115210A128A1100300A1254
:1003AC008A1564270A128A114830A6000030A7006B
:1003BC000A128A114C250A128A11A014E8298312F8
:1003CC000313A0108A290A128A1104288316031316
:1003DC001114F029831603131118F529F629F029A5
:1003EC00831603139112111783128C11C4309300CE
:0403FC00FF29831240
:1004000003138C1D042A052AFF29831203138C1160
:100410008316111B0C2A0F2A83128615112A8312A8
:10042000861183160313111783128C110130930068
:10043000192A831203138C1D1E2A1F2A192A8312BC
:1004400003138C118316111B262A292A8312861561
:100450002B2A831286118316031311171115302AC4
:10046000831603131119352A362A302A83160313EB
:1004700011143A2A8316031311183F2A402A3A2AE4
:1004800083160313911283128C11C5309300482AEE
:10049000831203138C1D4D2A4E2A482A83120313FC
:1004A0008C1183169115542A83160313141C592A90
:1004B0005A2A542A831203131308A1008316111613
:1004C000612A83160313111A662A672A612A831682
:1004D000031311156B2A831603131119702A712A3D
:1004E0006B2A8312031386152108762A03138312BD
:1004F00008008316031311147D2A831603131118A1
:10050000822A832A7D2A83160313911211178312DC
:100510008C11C43093008C2A831203138C1D912AF2
:10052000922A8C2A831203138C118316111B992A89
:100530009C2A831286159E2A831286118316031322
:10054000111783128C119301A52A831203138C1D9A
:10055000AA2AAB2AA52A831203138C118316111B16
:10056000B22AB52A83128615B72A831286118316FA
:100570000313111783128C119301BE2A83120313E4
:100580008C1DC32AC42ABE2A831203138C1183161E
:10059000111BCB2ACE2A83128615D02A83128611EC
:1005A00083160313111783128C119301D72A831218
:1005B00003138C1DDC2ADD2AD72A831203138C1126
:1005C0008316111BE42AE72A83128615E92A83126F
:1005D000861183160313111783128C1105309300B3
:1005E000F12A831203138C1DF62AF72AF12A8312AB
:1005F00003138C118316111BFE2A012B83128615FF
:10060000032B8312861183160313111783128C1187
:10061000033093000B2B831203138C1D102B112B13
:100620000B2B831203138C118316111B182B1B2BFE
:10063000831286151D2B831286118316031311173F
:1006400083128C114F309300252B831203138C1DC2
:100650002A2B2B2B252B831203138C118316111B92
:10066000322B352B83128615372B83128611831676
:100670000313111783128C114B3093003F2B8312FD
:1006800003138C1D442B452B3F2B831203138C111A
:100690008316111B4C2B4F2B83128615512B831263
:1006A000861183160313111783128C119301582B93
:1006B000831203138C1D5D2B5E2B582B83120313A7
:1006C0008C118316111B652B682B831286156A2BE0
:1006D0008312861183160313111711156F2B8316BE
:1006E00003131119742B752B6F2B8316031311141D
:1006F000792B8316031311187E2B7F2B792B8316EE
:1007000003139112111783128C11C4309300882B9C
:10071000831203138C1D8D2B8E2B882B83120313B6
:100720008C118316111B952B982B831286159A2BEF
:100730008312861183160313111783128C119301F0
:10074000A12B831203138C1DA62BA72BA12B831285
:1007500003138C118316111BAE2BB12B831286153C
:10076000B32B8312861183160313111783128C1176
:1007700040309300BB2B831203138C1DC02BC12B65
:10078000BB2B831203138C118316111BC82BCB2B8D
:1007900083128615CD2B831286118316031311172E
:1007A0001115D22B831603131119D72BD82BD22B4B
:1007B00003138312080083120313A9018316111473
:1007C0008312AA00E32B831603131118E82BE92BDD
:1007D000E32B831603139112111783128C11C4306B
:1007E0009300F22B831203138C1DF72BF82BF22BA3
:1007F000831203138C118316111BFF2B022C8312FF
:100800008615042C83128611831603131117831285
:100810008C1193010B2C831203138C1D102C112CA3
:100820000B2C831203138C118316111B182C1B2CF9
:10083000831286151D2C831286118316031311173C
:1008400083128C119301242C831203138C1D292CE9
:100850002A2C242C831203138C118316111B312C88
:10086000342C83128615362C8312861183160313BB
:10087000111783128C112A0893003E2C8312031344
:100880008C1D432C442C3E2C831203138C11831695
:10089000111B4B2C4E2C83128615502C8312861163
:1008A00083160313111783128C1125089300582CFB
:1008B000831203138C1D5D2C5E2C582C83120313A2
:1008C0008C118316111B652C682C831286156A2CDB
:1008D0008312861183160313111783128C112608B5
:1008E0009300722C831203138C1D772C782C722C9E
:1008F000831203138C118316111B7F2C822C8312FD
:100900008615842C83128611831603131117B02CBD
:10091000831203138C1129082707C6002808C70073
:1009200046080318C70A0A128A1113200A128A11EC
:100930009300A90A9B2C831203138C1DA02CA12CBD
:100940009B2C831203138C118316111BA82CAB2C28
:1009500083128615AD2C831286118316031311178B
:100960008312031329082707C6002808C700460872
:100970000318C70A0A128A1113200A128A110038B2
:10098000031DC32CC42C882C831203138C119301D8
:10099000C92C831203138C1DCE2CCF2CC92C83128F
:1009A00003138C118316111BD62CD92C8312861598
:1009B000DB2C831286118316031311171115E02CFB
:1009C000831603131119E52CE62CE02C8316031370
:1009D0001114EA2C831603131118EF2CF02CEA2CB7
:1009E000831603139112111783128C11C4309300D4
:1009F000F92C831203138C1DFE2CFF2CF92C83126F
:100A000003138C118316111B062D092D83128615D5
:100A10000B2D8312861183160313111783128C1169
:100A20009301122D831203138C1D172D182D122DD7
:100A3000831203138C118316111B1F2D222D831279
:100A40008615242D83128611831603131117831222
:100A50008C11403093002C2D831203138C1D312DEB
:100A6000322D2C2D831203138C118316111B392D5B
:100A70003C2D831286153E2D831286118316031397
:100A800011171115432D831603131119482D492DE4
:100A9000432D031383120800283083120313B90077
:100AA000C0012508BB00A12F831203133A08253A81
:100AB00003195B2D5C2D642DC00A3A080A128A15B1
:100AC000DD270A128A11A12FFF3083120313BD0004
:100AD000C101BC01742F83120313B9080319712DCE
:100AE000722D762D3908840083138001831203133D
:100AF0004008C32F023083120313BB073B0284005C
:100B000083130008C1006A2D83120313BC0A902DC1
:100B1000083083120313BD07FE3083120313BD0791
:100B2000023083120313BB073B02840083130008C7
:100B3000BE00840A0008BF003C1C9F2DA02DAF2DD5
:100B4000BF1FA32DA42DAB2DBE09BF09BE0A0319DB
:100B5000BF0AC103AE2D83120313BC01B22D831251
:100B60000313BC010B3083120313BD07831203135D
:100B70003D08F200F3013F08F1003E08F0000A12C0
:100B80008A11C6270A128A117008BA003D08F200BD
:100B9000F3013E08F0003F08F1000A128A11C6274F
:100BA0000A128A117408BE007508BF00C201C20A89
:100BB000C301ED2D831203133D08F200F301420837
:100BC000F0004308F1000A128A1584270A128A11DC
:100BD0007408C2007508C300C103831203134308DD
:100BE0003F02031DF52D42083E020318F82DF92D92
:100BF000DA2D032E83120313C00A20300A128A153D
:100C0000DD270A128A1183120313C1034108803AB7
:100C10007F3E03180C2E0D2EFA2D831203133C1C5D
:100C2000122E132E1A2EC00A2D300A128A15DD2715
:100C30000A128A114B2E831203134308F300420851
:100C4000F2003F08F1003E08F0000A128A11C627A0
:100C50000A128A117408F0007508F1003D08F200CC
:100C6000F3010A128A11C6270A128A117008C100FC
:100C70004108803A763E031C3E2E3F2E412E07301F
:100C8000C10783120313C00A4108303E0A128A15B5
:100C9000DD270A128A11831203133D08F200F301C3
:100CA0004208F0004308F1000A128A11C6270A120E
:100CB0008A117408C2007508C30043084204031D6A
:100CC000622E632E1B2E0A30831203133A02031C7A
:100CD0006A2E6B2E6D2E0730BA0783120313C00ADB
:100CE0003A08303E0A128A15DD270A128A11A12F0E
:100CF000832E83120313C00A20300A128A15DD27BF
:100D00000A128A11C103831203134108803A7E3EFE
:100D100003188B2E8C2E792E023083120313BB07FF
:100D20003B02840083130008BA00C00A3A080A1282
:100D30008A15DD270A128A11A12F023083120313AC
:100D4000BB073B02840083130008C200840A00082A
:100D5000C300BA01AE2E83120313BA0A831203131F
:100D60003A084207C6004308C70046080318C70AE6
:100D70000A128A1113200A128A110038031DC12E8B
:100D8000C22EAB2E831203133D083A020318C92E5C
:100D9000CA2ECC2E3A08BD00D72E83120313C00AE8
:100DA00020300A128A15DD270A128A11C103831224
:100DB00003133D08C11BE22EFF3A41070318E12E41
:100DC000E22ECD2EF82E831203134308C7004208EB
:100DD0000A128A1113200A128A11BA00C20A0319D0
:100DE000C30AC00A3A080A128A15DD270A128A11B4
:100DF00083120313BD033D0FFE2EFF2EE32EA12F02
:100E0000831203132708C70026080A128A11132029
:100E10000A128A112A3A031D0E2F0F2F1A2F0230A1
:100E2000BB073B02840083130008BD00A60A031918
:100E3000A70A4D2F831203132708C70026080A129A
:100E40008A1113200A128A11D03EBD00A60A031986
:100E5000A70A2708C70026080A128A1113200A12B7
:100E60008A11BA0030303A02031C3D2F372F3A3036
:100E70003A0203183D2F3C2F3F2F3E2F4D2F0A30B3
:100E8000F1003D080A128A1558270A128A113A07FA
:100E9000D03EBD00A60A0319A70A6A2D303083127E
:100EA00003133A02031C5B2F552F3A303A02031802
:100EB0005B2F5A2F5D2F5C2F692F0A30F1004108FC
:100EC0000A128A1558270A128A113A07D03EC10021
:100ED0006A2D83120313C00A3A080A128A15DD2705
:100EE0000A128A11A12FA12F831203132708C7000A
:100EF0002608A60A0319A70A0A128A1113200A1241
:100F00008A11BA00003A03196B2D2A3A03197A2D77
:100F1000043A0319002F763A0319882D3B3A031936
:100F2000782E073A0319842D0B3A03198C2D1C3A9D
:100F300003199D2E063A0319902D0D3A0319882D99
:100F40004E2F831203132708C7002608A60A031989
:100F5000A70A0A128A1113200A128A11BA00BA08C3
:100F6000031DB32FB42F542D83120313B908031993
:100F7000BA2FBB2FBF2F390884008313800183123F
:100F800003134008C32F031383120800F601F40172
:100F9000F50172087304031DD02FF001F101003434
:100FA0001F30F6040310F60AF20DF30D031CD32FC5
:100FB000F30CF20C73087102031DE02F720870022B
:100FC000031CE82F7208F0027308031C730AF10275
:100FD000F40DF50DF60BF61AD82FF61FF42FF409C1
:100FE000F40A0319F503F5097408F2007508F30013
:100FF000761F0034F009F00A0319F103F1090034F7
:101EB000F0000030711870070310F00D0310F10CE2
:101EC000F108031908005A2F831203138511A50086
:101ED0002508803E0A128A15BB270A128A150313A9
:101EE0008312080083120313851101300A128A1528
:101EF000BB270A128A1502300A128A1599270A127C
:101F00008A15031383120800F401F5010310F30C82
:101F1000F20C031C922F7008F40771080318710A61
:101F2000F5070310F00DF10D720873040319003466
:101F3000862F83120313A700043083120313A60015
:101F4000533083120313A800A62FA62F8312031366
:101F5000A80BAB2FAC2FA52F83120313A60BB12F09
:101F6000B22FA02F83120313A70BB72FB82F9C2FCC
:101F700003138312080083120313A600260E0F39E1
:101F8000F0000808F03970048800851485102608D0
:101F90000F39F0000808F0397004880085148510A6
:101FA0000D30A700D42FD42F83120313A70BD92FE2
:101FB000DA2FD32F0313831208008312031385151E
:101FC000C400440E0F39F0000808F039700488008E
:101FD0008514851044080F39F0000808F0397004A2
:101FE0008800851485100D30C500F72FF72F831258
:101FF0000313C50BFC2FFD2FF62F031383120800CC
:02400E00393542
:00000001FF
